:0200000480007A
:100000006F008004732F2034930F80006308FF0378
:10001000930F90006304FF03930FB0006300FF038E
:10002000130F000063040F0067000F00732F2034CC
:1000300063540F006F00400093E19153171F0000BD
:1000400023223FFC6FF09FFF93000000130100008C
:10005000930100001302000093020000130300004C
:100060009303000013040000930400001305000034
:10007000930500001306000093060000130700001C
:100080009307000013080000930800001309000004
:1000900093090000130A0000930A0000130B0000EC
:1000A000930B0000130C0000930C0000130D0000D4
:1000B000930D0000130E0000930E0000130F0000BC
:1000C000930F0000732540F16310050097020000B4
:1000D000938202017390523073500018970200000F
:1000E00093824202739052309B021000939252030B
:1000F0009382F2FF7390023B9302F0017390023AF5
:100100007350403097020000938242017390523046
:10011000735020307350303093010000970200007C
:10012000938282EE73905230130510001315F5017F
:10013000635C05000F00F00F930110009308D005D9
:10014000130500007300000093020000638A0200A0
:1001500073905210B7B200009B82921073902230BD
:100160007350003097020000938242017390123462
:10017000732540F173002030930000001B870000BE
:100180009303000093012000631C77269300100066
:100190001B87100093032000930130006312772621
:1001A000930030001B8770009303A0009301400070
:1001B00063187724930000001B870080930300805E
:1001C00093015000631E7722B70000801B87000058
:1001D000B70300809301600063147722B7000080AA
:1001E0001B870080B70300809B830380930170000E
:1001F00063187720930000001B87F07F9303F07F44
:1002000093018000631E771EB70000809B80F0FF83
:100210001B870000B70300809B83F3FF93019000CE
:100220006310771EB70000809B80F0FF1B87F07F74
:10023000B70300809B83E37F9301A0006312771CC8
:10024000B70000801B87F07FB70300809B83F37F9C
:100250009301B0006316771AB70000809B80F0FF0F
:100260001B870080B7F3FF7F9B83F37F9301C00060
:1002700063187718930000001B87F0FF9303F0FFCB
:100280009301D000631E77169300F0FF1B871000C8
:10029000930300009301E000631477169300F0FFCE
:1002A0001B87F0FF9303E0FF9301F000631A7714BC
:1002B000B70000809B80F0FF1B871000B703008011
:1002C00093010001631E77129300D0009B80B00061
:1002D00093038001930110016394701213020000D4
:1002E0009300D0001B87B000130307001302120015
:1002F00093022000E31652FE930380019301200134
:1003000063107310130200009300D0001B87A0003D
:1003100013000000130307001302120093022000D1
:10032000E31452FE9303700193013001631A730CBE
:10033000130200009300D0001B8790001300000000
:1003400013000000130307001302120093022000A1
:10035000E31252FE93036001930140016312730A9A
:10036000130200009300D0001B87B000130212009C
:1003700093022000E31852FE930380019301500181
:1003800063107708130200009300D00013000000F0
:100390001B87A0001302120093022000E31652FEF6
:1003A0009303700193016001631C77041302000042
:1003B0009300D00013000000130000001B87900082
:1003C0001302120093022000E31452FE9303600113
:1003D00093017001631677029B00000293030002F1
:1003E00093018001639E7000930010021B80200324
:1003F00093030000930190016314700063103002B6
:100400000F00F00F638001009391110093E1110040
:100410009308D00513850100730000000F00F00F52
:10042000930110009308D00513050000730000002D
:0C043000731000C000000000000000007D
:1010000000000000000000000000000000000000E0
:1010100000000000000000000000000000000000D0
:1010200000000000000000000000000000000000C0
:1010300000000000000000000000000000000000B0
:081040000000000000000000A8
:040000058000000077
:00000001FF
